:100000000C945D000C9485000C9485000C94850084
:100010000C9485000C9485000C9485000C9485004C
:100020000C9485000C9485000C9485000C9485003C
:100030000C9485000C9485000C9485000C9485002C
:100040000C943B030C9485000C9409030C94E3027C
:100050000C9485000C9485000C9485000C9485000C
:100060000C9485000C9485000000000024002700FB
:100070002A0000000000250028002B0004040404CE
:100080000404040402020202020203030303030342
:10009000010204081020408001020408102001021F
:1000A00004081020000000080002010000030407FB
:1000B0000000000000000000850311241FBECFEFE8
:1000C000D8E0DEBFCDBF11E0A0E0B1E0E4ECFAE0A3
:1000D00002C005900D92A035B107D9F722E0A0E546
:1000E000B1E001C01D92A137B207E1F710E0CDE504
:1000F000D0E004C02197FE010E945A05CC35D107FB
:10010000C9F70E94C4030C9460050C940000E1EB55
:10011000F0E02491EDE9F0E09491E9E8F0E0E49179
:10012000EE23C9F0222339F0233001F1A8F4213065
:1001300019F1223029F1F0E0EE0FFF1FEE58FF4FCA
:10014000A591B4912FB7F894EC91811126C09095A8
:100150009E239C932FBF08952730A9F02830C9F023
:10016000243049F7209180002F7D03C0209180002A
:100170002F7720938000DFCF24B52F7724BDDBCFEE
:1001800024B52F7DFBCF2091B0002F772093B000B6
:10019000D2CF2091B0002F7DF9CF9E2BDACFAF9236
:1001A000BF92CF92DF92EF92FF920F931F93CF9364
:1001B000DF936C017B018B01040F151FEB015E01C6
:1001C000AE18BF08C017D10759F06991D601ED915B
:1001D000FC910190F081E02DC6010995892B79F7FA
:1001E000C501DF91CF911F910F91FF90EF90DF90AC
:1001F000CF90BF90AF900895FC01538D448D252F73
:1002000030E0842F90E0821B930B541710F0CF96B0
:10021000089501970895FC01918D828D981761F0E2
:10022000A28DAE0FBF2FB11D5D968C91928D9F5FF9
:100230009F73928F90E008958FEF9FEF0895FC01D8
:10024000918D828D981731F0828DE80FF11D858D8B
:1002500090E008958FEF9FEF0895FC01918D228D1E
:10026000892F90E0805C9F4F821B91098F739927A3
:10027000089586E691E00E942D0121E0892B09F482
:1002800020E0822F089580E090E0892B29F00E94E1
:10029000390181110C9400000895FC01A48DA80F70
:1002A000B92FB11DA35ABF4F2C91848D90E00196B8
:1002B0008F739927848FA689B7892C93A089B189D8
:1002C0008C91837080648C93938D848D981306C079
:1002D0000288F389E02D80818F7D80830895EF92DD
:1002E000FF920F931F93CF93DF93EC0181E0888FF0
:1002F0009B8D8C8D98131AC0E889F989808185FFC0
:1003000015C09FB7F894EE89FF896083E889F98961
:1003100080818370806480839FBF81E090E0DF9163
:10032000CF911F910F91FF90EF900895F62E0B8DB6
:1003300010E00F5F1F4F0F731127E02E8C8D8E1171
:100340000CC00FB607FCFACFE889F989808185FFD8
:10035000F5CFCE010E944D01F1CFEB8DEC0FFD2FBB
:10036000F11DE35AFF4FF0829FB7F8940B8FEA8993
:10037000FB8980818062CFCFCF93DF93EC01888DA2
:100380008823B9F0AA89BB89E889F9898C9185FD10
:1003900003C0808186FD0DC00FB607FCF7CF8C919E
:1003A00085FFF2CF808185FFEDCFCE010E944D0108
:1003B000E9CFDF91CF9108953FB7F894809156012E
:1003C00090915701A0915801B091590126B5A89B71
:1003D00005C02F3F19F00196A11DB11D3FBFBA2FD7
:1003E000A92F982F8827BC01CD01620F711D811D97
:1003F000911D42E0660F771F881F991F4A95D1F71C
:100400000895AF92BF92CF92DF92EF92FF920F9337
:100410001F93CF93DF938B01D0E0C0E001975C0185
:100420008091670290916802DC01ED91FC9100845B
:10043000F185E02D0995A816B906ACF00E94DC0103
:100440006B017C010E94DC016C197D098E099F09FA
:10045000683E734081059105A8F321960C171D078E
:10046000F9F680E001C081E0DF91CF911F910F91FB
:10047000FF90EF90DF90CF90BF90AF900895DC0198
:10048000ED91FC910190F081E02D0994CF92DF92E3
:10049000EF92FF920F931F93CF93DF9300D000D082
:1004A000CDB7DEB78C01FC0101900020E9F7319750
:1004B000E81BF90B87E080935A01E0935B011092EF
:1004C0005C0110925D0180915A0190915B01A091B5
:1004D0005C01B0915D0189839A83AB83BC836CEF2F
:1004E0007FEF80916702909168020E943F02CE01E7
:1004F00001967C016E0195E0C90ED11C80916702C6
:1005000090916802D7016D917D01DC01ED91FC9124
:100510000190F081E02D0995EC14FD0479F76DEF61
:100520007FEF80916702909168020E943F026EEF18
:100530007FEF80916702909168020E943F02F12C48
:100540002F2D30E0F80101900020E9F73197E01BF2
:10055000F10B80916702909168022E173F0758F4C3
:10056000200F311FF9016081062E000C770B0E94CD
:100570003F02F394E5CF6FEF7FEF0F900F900F9056
:100580000F90DF91CF911F910F91FF90EF90DF902F
:10059000CF900C943F0280915001882369F0109213
:1005A000500180E00E94870080915001882341F033
:1005B00082E191E00C94460281E080935001F2CFF9
:1005C00080E391E0F7CF1F920F920FB60F921124A4
:1005D0002F933F934F935F936F937F938F939F934B
:1005E000AF93BF93EF93FF9386E691E00E944D0196
:1005F000FF91EF91BF91AF919F918F917F916F91FB
:100600005F914F913F912F910F900FBE0F901F90D0
:1006100018951F920F920FB60F9211242F938F935C
:100620009F93EF93FF93E0917601F09177018081A2
:10063000E0917C01F0917D0182FD1BC09081809151
:100640007F018F5F8F7320918001821741F0E091CD
:100650007F01F0E0EA59FE4F958F80937F01FF9173
:10066000EF919F918F912F910F900FBE0F901F9040
:1006700018958081F4CF1F920F920FB60F9211241C
:100680002F933F938F939F93AF93BF93809152018A
:1006900090915301A0915401B091550130915101B5
:1006A00023E0230F2D3758F50196A11DB11D20938E
:1006B00051018093520190935301A0935401B09340
:1006C00055018091560190915701A0915801B09128
:1006D00059010196A11DB11D8093560190935701B8
:1006E000A0935801B0935901BF91AF919F918F9101
:1006F0003F912F910F900FBE0F901F90189526E8F5
:10070000230F0296A11DB11DD2CFE6E6F1E01382C0
:10071000128288EE93E0A0E0B0E084839583A68304
:10072000B78384E091E09183808385EC90E09587A6
:10073000848784EC90E09787868780EC90E0918BAB
:10074000808B81EC90E0938B828B82EC90E0958B98
:10075000848B86EC90E0978B868B118E128E138E95
:10076000148EF0936802E0936702EEE5F1E089E908
:10077000808387E1818384E3828381E083831482A1
:100780001582168217820895CF93DF93CDB7DEB717
:100790002C970FB6F894DEBF0FBECDBF789484B50A
:1007A000826084BD84B5816084BD85B5826085BD6D
:1007B00085B5816085BD80916E00816080936E00FB
:1007C00010928100809181008260809381008091ED
:1007D000810081608093810080918000816080939E
:1007E00080008091B10084608093B1008091B0005E
:1007F00081608093B00080917A00846080937A0059
:1008000080917A00826080937A0080917A00816082
:1008100080937A0080917A00806880937A001092A9
:10082000C100E0917601F091770182E08083E09150
:100830007601F09177011082E0917201F0917301DD
:100840001082E0917401F091750180E18083109233
:100850007E01E0917A01F0917B0186E08083E09156
:100860007801F0917901808180618083E091780145
:10087000F0917901808188608083E0917801F09126
:100880007901808180688083E0917801F09179011D
:1008900080818F7D8083EDE9F0E02491E9E8F0E04C
:1008A0008491882399F090E0880F991FFC01E85902
:1008B000FF4FA591B491FC01EE58FF4F85919491A3
:1008C0008FB7F894EC91E22BEC938FBF809162018B
:1008D0008260809362018BEC92E090936C02809333
:1008E0006B026E018DE0C80ED11C90E0E92E90E005
:1008F000F92E8091670290916802DC01ED91FC91E4
:100900000084F185E02D0995892B09F450C0809170
:10091000670290916802DC01ED91FC910284F385FD
:10092000E02D09958C3F09F042C064E670E085E057
:1009300090E00E9401028823D1F18E01075F1F4FD2
:1009400058018091670290916802DC01ED91FC9161
:100950000284F385E02D0995F80181938F01EC1550
:10096000FD0579F78091670290916802DC01ED91B5
:10097000FC910284F385E02D099589853A852B85C4
:100980009C8580935A0130935B0120935C01909386
:100990005D01833009F476C0B0F4813009F446C0BB
:1009A000E0916902F0916A02823009F46FC0E114AB
:1009B000F10409F49ECF0E943901882309F499CFEC
:1009C0000E94000096CF843009F462C0853079F728
:1009D00080905B01082D10E062E370E0C801029690
:1009E0000E940102882319F38091670290916802A6
:1009F000DC01ED91FC910284F385E02D099583E003
:100A0000A82E82E0B82E912C809167029091680206
:100A1000DC01ED91FC910284F385E02D8914E9F16C
:100A20000995F50181935F019394EECF88E0EEE59F
:100A3000F1E0DE01119601900D928A95E1F76EEFDB
:100A40007FEF80916702909168020E943F028E01C1
:100A50000F5F1F4FF80161918F01062E000C770B7D
:100A600080916702909168020E943F02A016B10631
:100A700089F76FEF7FEF80916702909168020E9483
:100A80003F0295CFE0916B02F0916C0209958FCFF8
:100A9000E0916D02F0916E02F9CF0995F801ED5FDA
:100AA000FD4F1082E0916F02F091700283E092E0BE
:100AB00009957DCFEE0FFF1F0590F491E02D09946D
:040AC000F894FFCFD8
:100AC400000000006F01CF00FC00BC012D010B01F0
:100AD4001F017075626C6973682074656C652F6D95
:100AE40079746F7069632F706F776572206F6E0011
:100AF4007075626C6973682074656C652F6D7974A8
:100B04006F7069632F706F776572206F666600007F
:00000001FF
